:1000000000308A003A280000831A0A28A500030E4F
:10001000A6000F288312A500030EA600A6140A0846
:10002000AD008A018313A50E0408A7002008A800CC
:100030002108A9002208AA002308AB002408AC006C
:1000400083128B1D25280B184228270884002808B6
:10005000A0002908A1002A08A2002B08A3002C0850
:10006000A4002D088A00260E83008312250EA618F0
:100070008316090007308A00FF278316900000309E
:100080008A00D1280508B0000B108A1125282F30CE
:1000900084000008031959280230A100A001A00B18
:1000A0004F28A10B4E289730A000A00B5528800B9D
:1000B0004C2800342E10003085190130003A031D01
:1000C00073280A30AF004720003085190130003A0C
:1000D000031D7328003085190130013C031D712870
:1000E00072286A282E1400302E180130A1001B2916
:1000F000AE012E080F3C031C8C2805150930A0000A
:10010000A00B80280000000005110730A000A00B04
:1001100087280000AE0A792800342F3084000310AD
:10012000800C00080319982896280000800B952859
:10013000003478200730AF0047200230AE009E30F8
:10014000AF008D20AE0B9F28782021292E10003083
:10015000051A0130003A031DBF280A30AF004720BE
:100160000030051A0130003A031DBF280030051A7F
:100170000130013C031DBD28BE28B6282E140030D6
:100180002E180130A100222978200530AF00472029
:100190000230AE00AD30AF008D20AE0BCA28782003
:1001A000282984011F30830583161F08F0399F001A
:1001B00083121F1307309F00703083168F0070303A
:1001C0008F00183065009501811707308312990060
:1001D0008316050806308312A000A00BED2800004E
:1001E00019088C1183161F080F399F0083121F08EE
:1001F0000C399F0083161F08F0399F0083121F13CC
:10020000831605108312051083168510831285103E
:100210008316051183120511831685128312851228
:100220008B158316961583128B1583161616C03000
:1002300083128B045A28210B21290A30AF00472052
:100240009928A628210B28290A30AF004720C42866
:100250008B158316961583128B158316161663005D
:10026000000083128B118316961183128B11831653
:08027000161283121A29630023
:020FFE000034BD
:02400E00C43CB0
:00000001FF
